:100000000C9477000C949F130C94C6130C949F00CF
:100010000C949F000C949F000C949F000C949F00E4
:100020000C949F000C949F000C949F000C949F00D4
:100030000C949F000C947F080C949F000C949F00DC
:100040000C94ED130C949F000C94B1160C94E316D1
:100050000C949F000C949F000C949F000C949F00A4
:100060000C949F000C949F003B4D433D003B4D552D
:100070003D004D533D00556E737570706F72746521
:100080006420636F6D6D616E640020557365206F31
:100090006E65206F6620000000000800020100006D
:1000A0000304070000000000000000010204081023
:1000B00020408001020408102001020408102004DE
:1000C00004040404040404020202020202030303FF
:1000D00003030300000000250028002B000000009F
:1000E00000240027002A0000190813175C081124B7
:1000F0001FBECFEFD8E0DEBFCDBF12E0A0E0B1E081
:10010000E6EFF6E402C005900D92A631B107D9F7EB
:1001100024E0A6E1B2E001C01D92AB3AB207E1F7DC
:1001200010E0CCEED0E004C02297FE010E949A1DA0
:10013000C83ED107C9F70E9457170C946E230C9440
:100140000000CF92DF92EF92FF920F931F930E94D5
:10015000431400911D0210911E0220911F02309144
:1001600020026B017C01C01AD10AE20AF30A97014E
:10017000860160931D0270931E0280931F0290936C
:1001800020020A3511052105310578F181E0C816F4
:100190008DE7D806E104F10410F4960102C021E0D5
:1001A0003DE74A9B03C03195219531098091620357
:1001B0008B34D8F4809162038F5F809362038091C7
:1001C0006303609161030E94421D90936303E09179
:1001D0006303F0E0EE0FFF1FEB59FC4F31832083E8
:1001E000809163038F5F809363031F910F91FF9052
:1001F000EF90DF90CF9008950F931F9360912702A7
:100200008DE00E943615109227020E94431400913F
:100210001D0210911E0220911F0230912002601BCE
:10022000710B820B930B62307D478105910520F0A5
:100230001F910F910C94A1001F910F91089581E2DD
:1002400092E00E94FF188BE593E00E94FF1885E57D
:1002500093E00C94FF18CF93DF93EC01FB01248112
:1002600035810E94421BCE01DF91CF91089541E07C
:1002700050E061EA70E080E00C946D1380E00C9433
:100280008D13CF93DF931F92CDB7DEB72B9A2091BA
:10029000060130910701482F429FC001439F900DF6
:1002A000112469830E948E142B98809106019091ED
:1002B00007016981FC016E9FC0016F9F900D1124A1
:1002C0000F90DF91CF910C948E14EF92FF920F93C9
:1002D0001F93CF93DF93F82EE92E0E943E0100E09A
:1002E00010E02091080130E0021713072CF56FE1B0
:1002F00081E00E944101CF2DDE2D29912223C9F0FA
:10030000213371F0263449F02033B9F763E081E0FE
:100310000E94410163E081E009C063E081E002C026
:1003200061E083E00E94410161E083E00E944101BD
:10033000E4CF0F5F1F4FD5CFDF91CF911F910F916A
:10034000FF90EF900C9437013F924F925F926F9223
:100350007F928F929F92AF92BF92CF92DF92EF9255
:10036000FF920F931F93CF93DF93082FEB01542E2F
:10037000452E59010E9443146B017C0110E0812C31
:10038000912CB401600F711FC617D707A8F1C501E2
:100390000E94FA1A8053E52DF42DE80FF11DE80FA5
:1003A000F11D90818181382E331C3324331C692E3A
:1003B000782E31F077FE0CC071946194710808C0FA
:1003C00077FE03C071946194710888E1681A71081E
:1003D0000E9443146C157D058E059F05C8F33320DC
:1003E00011F02B9801C02B9AC60CD71CE11CF11CF4
:1003F0008FEF881A980AC5CF0E9443146C157D05AB
:100400008E059F05C8F3DF91CF911F910F91FF904B
:10041000EF90DF90CF90BF90AF909F908F907F90A4
:100420006F905F904F903F9008954F925F926F92C0
:100430007F928F929F92AF92BF92CF92DF92EF9274
:10044000FF920F931F93CF93DF93982E862E2A014E
:100450002B9A0E9443146B017C01662457FC609424
:10046000762C891408F446C0692D70E081E292E090
:100470000E94FA1A90ED980F9A3010F4892F01C05B
:100480008753C4E0D0E008E0A82EBB24A7FCB094BA
:100490000E9443146C157D058E059F05C8F310E07E
:1004A00098012A213B21232B71F02B98C40CD51CD9
:1004B000E61CF71C0E9443146C157D058E059F05F4
:1004C000C8F32B9A0DC02B9AC40CD51CE61CF71C44
:1004D0000E9443146C157D058E059F05C8F32B986B
:1004E000C40CD51CE61CF71C15950795219781F6C1
:1004F0009394B7CF0E9443146C157D058E059F051C
:10050000C8F3DF91CF911F910F91FF90EF90DF9093
:10051000CF90BF90AF909F908F907F906F905F90A3
:100520004F900895CF92DF92EF92FF920F931F9317
:10053000CF93DF9300D000D000D0CDB7DEB78C01D1
:100540006B01FC01E080F1806DE071E0CE0101966D
:100550000E946D19A701BE016F5F7F4F81E292E09B
:100560000E94261B7C01CE0101960E94FF18FFEF1E
:10057000EF16FF0601F1F801408151814F3FFFEF77
:100580005F07C9F0970161E272E0CE0101960E9417
:10059000421BBE016F5F7F4FC6010E94B919CE0199
:1005A00001960E94FF188FEFE81AF80AF801F1820D
:1005B000E08281E001C080E026960FB6F894DEBFAD
:1005C0000FBECDBFDF91CF911F910F91FF90EF90A4
:1005D000DF90CF900895BF92CF92DF92EF92FF927B
:1005E0000F931F93CF93DF93CDB7DEB7C856D109D2
:1005F0000FB6F894DEBF0FBECDBF67E072E0CE014C
:100600008F599F4F0E946D196EE170E0CE018F5996
:100610009F4F0E943019A9961FAE1EAEA9970E9447
:100620003E011FEF01E042E1F42E59E0E52E62E0C9
:10063000D62ECC24C394BE016F597F4FCE01895969
:100640009F4F0E949202882309F44FC060E070E03F
:10065000CE018F599F4F0E94FA1A833589F561E0C8
:1006600070E0CE018F599F4F0E94FA1A833419F31C
:1006700061E070E0CE018F599F4F0E94FA1A8D34CD
:1006800059F41F5FE1E0F0E0EC0FFD1FF19EE00D7B
:10069000F11D1124C282CFCF61E070E0CE018F59ED
:1006A0009F4F0E94FA1A823531F61F5FE1E0F0E0B9
:1006B000EC0FFD1FF19EE00DF11D1124D282BBCF86
:1006C00060E070E0CE018F599F4F0E94FA1A80358A
:1006D00009F068C062E070E0CE018F599F4F0E9420
:1006E000FA1A8D3309F05EC082C0B12C32E1C32EFC
:1006F000B016D1F1D12CED2CF12CCE9CA001CF9CC9
:10070000500D1124E1E0F0E0EC0FFD1FE40FF51FA8
:100710008281823079F44A5F5F4F21E030E02C0F14
:100720003D1F420F531F6481758121E232E08381B6
:100730000E94A401CE9CF001CF9CF00D112481E019
:1007400090E08C0F9D1FE80FF91F8281813031F4FA
:1007500040815181648183810E9415022B98D3943A
:100760001D1548F6B394C4CF0E94370161E272E0D0
:100770008AE094E00E94F217CE018F599F4F0E94A9
:10078000FF18C859DF4F0FB6F894DEBF0FBECDBFBC
:10079000DF91CF911F910F91FF90EF90DF90CF905D
:1007A000BF90089560E070E0CE018F599F4F0E9486
:1007B000FA1A823509F050C061E070E0CE018F591D
:1007C0009F4F0E94FA1A8D3309F046C042E050E074
:1007D000BE016F597F4FCE01855A9F4F0E942B015A
:1007E000CE01855A9F4F0E94871B062F82C022E0B0
:1007F00030E041E050E0BE016F597F4FCE01855A95
:100800009F4F0E94421BCE01855A9F4F0E94871B1B
:10081000B62ECE01855A9F4F0E94FF1843E050E04C
:10082000BE016F597F4FCE01855A9F4F0E942B0109
:10083000CE01855A9F4F0E94871BE19EF001112433
:10084000EB0DF11D3396EE0FFF1F21E030E02C0F72
:100850003D1FE20FF31F4BC060E070E0CE018F59E7
:100860009F4F0E94FA1A8434B9F4A9968EAD9FADB9
:10087000A997E1E0F0E0EC0FFD1FF19EE00DF11D06
:10088000112421E0280FA6963FADA697231B2383B2
:10089000029795838483CFCE60E070E0CE018F59BC
:1008A0009F4F0E94FA1A833409F0C5CE61E070E0D0
:1008B000CE018F599F4F0E94FA1A8D3309F0BBCE9B
:1008C00042E050E0BE016F597F4FCE01855A9F4FE5
:1008D0000E942B01CE01855A9F4F0E94871BE1E0A9
:1008E000F0E0EC0FFD1FF19EE00DF11D112471836E
:1008F0006083CE01855A9F4F0E94FF189CCE62E70D
:1009000070E08AE094E00E94A41760912B0270E0EE
:100910004AE050E08AE094E00E94B9186DE670E089
:100920008AE094E00E94A4176091290270E04AE0F6
:1009300050E08AE094E00E94B91868E670E08AE02E
:1009400094E00E94A41760912A0270E04AE050E00F
:100950008AE094E00C94C118CF93DF93CDB7DEB753
:10096000AE970FB6F894DEBF0FBECDBF61E070E06A
:1009700081E292E00E94FA1A843729F161E070E086
:1009800081E292E00E94FA1A823721F542E050E0BB
:1009900061E272E0CE0101960E942B0120E030E07E
:1009A00043E050E0BE01675D7F4FCE0101960E949B
:1009B000FC1ACE0101960E94FF18CE0189960E9472
:1009C0008F1F8093080161E272E08AE094E00E9448
:1009D000F21795C061E070E081E292E00E94FA1A9D
:1009E0008337F1F42B9A42E050E061E272E0CE01ED
:1009F00089960E942B0120E030E048E250E0BE01E1
:100A00006F5F7F4FCE0189960E94FC1ACE018996B6
:100A10000E94FF18CE0101960E9465012B98D3CF4A
:100A200061E070E081E292E00E94FA1A8336A9F454
:100A300042E050E061E272E0CE0101960E942B019B
:100A4000CE0101960E94871B7093070160930601F7
:100A5000CE0101960E94FF18B6CF61E070E081E2FE
:100A600092E00E94FA1A803709F049C067E072E00C
:100A7000CE0189960E946D1964E170E0CE018996DD
:100A80000E9430196FE071E0CE0189960E94C5196D
:100A90004AE060910801CE0101960E94DD19BE0175
:100AA0006F5F7F4FCE0189960E94621ACE01019638
:100AB0000E94FF1867E971E0CE0189960E94691AC9
:100AC00060910601709107014AE0CE0101960E94F3
:100AD0000A1ABE016F5F7F4FCE0189960E94621A8B
:100AE000CE0101960E94FF18BE01675D7F4F8AE02C
:100AF00094E00E94F217CE0189960E94FF18AE96EC
:100B00000FB6F894DEBF0FBECDBFDF91CF91089531
:100B1000CF93DF9300D0CDB7DEB72091A7043091FB
:100B2000A8042115310511F42BEA34E0CE01019619
:100B3000821B930B0F900F90DF91CF910895CF926E
:100B4000DF92EF92FF920E9437146B017C0128EE36
:100B500033E040E050E00E94761D809118029091B1
:100B60001902A0911A02B0911B02C816D906EA0612
:100B7000FB0648F48091160290911702019690931B
:100B8000170280931602C0921802D0921902E092C6
:100B90001A02F0921B02CA01B901FF90EF90DF9098
:100BA000CF9008956AE171E08AE094E00E94041811
:100BB00061E070E080E090E00C94661461E070E029
:100BC00081E292E00E94FA1A813511F40E943E01FE
:100BD00061E070E081E292E00E94FA1A853411F43B
:100BE0000C9437010895262F220F330B94E049020D
:100BF000B0011124682B622B81E090E00C947322E9
:100C0000CF93DF9361E070E081E292E00E94FA1AF4
:100C1000873421F4DF91CF910C947F0462E070E07F
:100C200081E292E00E94FA1A833599F062E070E066
:100C300081E292E00E94FA1A853571F062E070E07C
:100C400081E292E00E94FA1A833441F4CAE2D2E0CF
:100C500005C0CBE2D2E002C0C9E2D2E061E070E0C0
:100C600081E292E00E94FA1A853419F481E08883C7
:100C700009C061E070E081E292E00E94FA1A8434D7
:100C800059F4188240912A026091290280912B0226
:100C9000DF91CF910C94F305DF91CF91089560E03F
:100CA00070E081E292E00E94FA1A803511F40C940F
:100CB000D20560E070E081E292E00E94FA1A8F3380
:100CC00009F072C06FE38AE094E00E94D5176AE8E9
:100CD00070E08AE094E00E94A41766E58AE094E060
:100CE0000E94D51760E28AE094E00E94D51769E679
:100CF0008AE094E00E94D51760E28AE094E00E94C6
:100D0000D51762E58AE094E00E94D51760E28AE098
:100D100094E00E94D51764E78AE094E00E94D5171A
:100D200060E28AE094E00E94D51768E58AE094E0EA
:100D30000E94D51760E28AE094E00E94D51766E42D
:100D40008AE094E00E94D51760E28AE094E00E9475
:100D5000D51763E58AE094E00E94D51760E28AE047
:100D600094E00E94D51760E58AE094E00E94D517D0
:100D700060E28AE094E00E94D51763E48AE094E0A0
:100D80000E94D51760E28AE094E00E94D51767E4DC
:100D90008AE094E00E94D51760E28AE094E00E9425
:100DA000D51767E072E00AC060E070E081E292E08F
:100DB0000E94FA1A863531F46DE171E08AE094E020
:100DC0000C94041860E070E081E292E00E94FA1A4C
:100DD000823549F40E9488054AE050E0BC018AE06F
:100DE00094E00C94C11860E070E081E292E00E940F
:100DF000FA1A893641F488E292E00E94E408892BCD
:100E000081F40C94AC0460E070E081E292E00E9416
:100E1000FA1A833561F488E292E00E94E408892B93
:100E200021F081E080931C0208950C94EB0260E0B5
:100E300070E081E292E00E94FA1A843751F40E9435
:100E40009F05AB01BC012AE030E08AE094E00C94FD
:100E5000ED1860E070E081E292E00E94FA1A8835B5
:100E600011F40C94DE0560E070E081E292E00E94F3
:100E7000FA1A8634D1F060E070E081E292E00E94DC
:100E8000FA1A833411F40C94000660E070E081E2F9
:100E900092E00E94FA1A873411F40C947F0466E7FA
:100EA00070E08AE094E00C94E01708951F93CF93CC
:100EB000DF9300D0CDB7DEB780911C02882389F084
:100EC00010921C020E944F0680911C02811106C0E4
:100ED00067E072E081E292E00E94C51981E08093B0
:100EE000270211E080916203882341F1809162031F
:100EF00081508093620380916403609161030E943A
:100F0000421D90936403E091640381E08E0F80930F
:100F10006403F0E0EE0FFF1FEB59FC4F80819181DD
:100F20009A838983BE016F5F7F4F88E292E00E94BF
:100F30004B138823B9F210932702D4CF0F900F9050
:100F4000DF91CF911F910895EF92FF920F931F931E
:100F5000CF93DF93EC017B018A0181E090E00E9456
:100F60006B22982F9170988381FB992790F9F70154
:100F7000908382FB882780F9F8018083DF91CF91ED
:100F80001F910F91FF90EF90089526E040E051EE01
:100F900060E070E08AE094E00E944F1660E082E03A
:100FA0000E94FD1461E08BE00E94FD1461E08DE081
:100FB0000E94FD1480E1809381001092800082E005
:100FC0008093FD0388E199E79093FF038093FE03EC
:100FD000909387008093860082E1809381008CEF5C
:100FE00090E09093FC038093FB0381E080936F007B
:100FF00080E090E00E946B228B3049F44AE252E09C
:1010000069E272E08BE292E00E94A4070AC06BE002
:1010100080E090E00E94732267E081E090E00E940F
:1010200073220E94370164E170E081E292E00C9447
:1010300030190F931F93CF93DF938BE48093610359
:10104000109262031092640310926303CBE3D3E027
:10105000D0934003C0933F030DE313E0109342038A
:101060000093410367E072E085E593E00E946D190B
:1010700067E072E08BE593E00E946D19F801118240
:1010800010821982188288E292E00E94A60867E026
:1010900072E081E292E00E946D190E944314609315
:1010A0001D0270931E0280931F0290932002DF9115
:1010B000CF911F910F9108950C941F01CF93C1E020
:1010C0008AE094E00E946C15892BB9F08AE094E0E4
:1010D0000E9485158A3041F01CF4882329F007C04E
:1010E0008D3011F0833219F4C0931C02E9CF682FC0
:1010F00081E292E00E94791AE3CFCF9108951F9286
:101100000F920FB60F9211242F933F934F935F933B
:101110006F937F938F939F93AF93BF93EF93FF93BF
:10112000E091FB03F091FC030995FF91EF91BF91D2
:10113000AF919F918F917F916F915F914F913F916F
:101140002F910F900FBE0F901F901895FC01E85F34
:10115000FE4F1082B39610827B97108231961182D7
:1011600010827B962FEF2083FC012083AC0120E0CE
:1011700030E0FA01E15EFE4F11821082FC01E20FC5
:10118000F31F14822F5F3F4F4E5F5F4F26303105B4
:1011900081F7FC01E55FFE4F1082339626E930E0CF
:1011A000318320833D964DEC5CEC6CE47EE3408320
:1011B00051836283738372971082339610823196C3
:1011C000108233971082089580E090E00895CF93C5
:1011D000DF93FC01E55DFE4FD081C0E07D97CD1728
:1011E000C1F0DC01A15EBE4F2D913C91AB01421BD1
:1011F000530B9A0157FF03C031952195310902968F
:10120000408151814217530714F08C2F03C0CF5FE8
:10121000E6CF8FEFDF91CF910895FC011482158204
:101220001682178210861186411104C0DC01A85F66
:10123000BE4F4C91641780F4DF01A60FB11D1A96C2
:101240008C91DF01A80FB11D14968C9114978F5FBC
:1012500014968C936F5FEECF08952F923F924F922A
:101260005F926F927F928F929F92AF92BF92CF9236
:10127000DF92EF92FF920F931F93CF93DF93CDB73F
:10128000DEB72E970FB6F894DEBF0FBECDBF9E8798
:101290008D8740E060E00E940D09ED85FE85E55DEB
:1012A000FE4F5080712C2D853E85255E3E4F3A873E
:1012B00029878D859E85885F9E4F9C878B877514B7
:1012C00009F4C3C044244394470C642C272C312CCC
:1012D000C101880F991FAD85BE858A0F9B1FFC0138
:1012E000E15EFE4FFA83E9832A0E3B1EF4E02F0EE7
:1012F000311C29813A8138872F83651409F4A3C0F2
:10130000862D90E09C838B83880F991F9E838D830D
:10131000FC01AD85BE85EA0FFB1FE15EFE4F00813B
:101320001181C80117FF04C088279927801B910BE2
:10133000BC01882777FD8095982F0E942B1CE9859A
:10134000FA8520813181428153810E94DF1C4B014B
:101350005C01A981BA81CD90DC907801EC18FD0880
:10136000F7FE03C0F194E194F10820E030E040E0A2
:101370005FE3C501B4010E94DF1C9B01AC01C50104
:10138000B4010E94941B0E94F81B6E157F050CF49B
:1013900058C0EB85FC85208180E090E0821750F4F6
:1013A000ED85FE85E80FF91F3285361101C0728682
:1013B0000196F4CFD1014C91552747FD5095EB8113
:1013C000FC812D853E85E20FF31FE481FF27E7FDB9
:1013D000F0959A012E0F3F1F21153105E1F4C49EAF
:1013E000C001C59E900DD49E900D1124B9010E949C
:1013F000621D7B010E9FC0010F9F900D1E9F900DDF
:101400001124B9010E94621DE60EF71EAF81B88556
:10141000ED92FC920CC00C0D1D1D17FF02C00F5F5A
:101420001F4F15950795E981FA8111830083ED819E
:10143000FE812D853E85E20FF31FE15EFE4F118296
:10144000108263945ACF742C3ACF2E960FB6F8942C
:10145000DEBF0FBECDBFDF91CF911F910F91FF90E7
:10146000EF90DF90CF90BF90AF909F908F907F9044
:101470006F905F904F903F902F9008953F924F92C2
:101480005F926F927F928F929F92AF92BF92CF9214
:10149000DF92EF92FF920F931F93CF93DF93EC01B4
:1014A0008FEF8883FE01E55DFE4F30806E0100E026
:1014B00010E0EE24EA94FE2C4E0188EF881A8EEF9D
:1014C000980A031508F06AC0F601E15EFE4F5F015D
:1014D000FFEFEF16FF0639F5F5018081918197FD49
:1014E00022C0FE01E00FF11F6481772767FD709530
:1014F000872F972F0E942B1C2B013C01F401608148
:1015000070E080E090E00E942B1C2BE734E14EE27B
:101510005EE30E94DF1C9B01AC01C301B2010E948B
:10152000DB1C1816A4F1F5012081318137FD30C094
:10153000C701880F991F8C0F9D1FFC01E15EFE4FB4
:1015400080819181281739071CF5FE01E00FF11FFA
:101550006481772767FD7095872F972F0E942B1C3A
:101560002B013C01F401608170E080E090E00E947A
:101570002B1C2BE734E14EE25EE30E94DF1C9B0153
:10158000AC01C301B2010E94DB1C18160CF47801F7
:101590000F5F1F4FF2E0CF0ED11C93CF8FEFE816F5
:1015A000F80641F0E882CF5EDE4F81E090E099835B
:1015B000888301C080E0DF91CF911F910F91FF9050
:1015C000EF90DF90CF90BF90AF909F908F907F90E3
:1015D0006F905F904F903F9008958F929F92AF923F
:1015E000BF92CF92DF92EF92FF920F931F93CF9310
:1015F000DF93FC018C010F5E1E4FD8018D919C91F1
:101600001197019709F07CC05A96BC90BA94C7E034
:10161000AC2E6F01B8EFCB1ABEEFDB0AB7FC70C07F
:101620002B2D332727FD3095C901880F991F8E0F69
:101630009F1FDC01A15EBE4FCD91DC91D7FF5EC044
:10164000D195C195D109C83682E4D80708F056C0B3
:10165000E080FF24E7FCF094C701880F991F8E0FEC
:101660009F1FDC01A15EBE4F8D909C90CE01B40106
:101670000E944E1D6832710508F040C0A89CC00150
:10168000A99C900D11248C179D07C0F5DF01A20FB6
:10169000B31F14968C9186308CF5D6014C9150E096
:1016A000BA0161507109912C892D90E08617970736
:1016B00084F4DF01A80FB91F1B96CC911B97D0E0D3
:1016C000C217D307C9F41A96AC91B0E0AE15BF05A6
:1016D00099F4485251098417950784F4DF01A45DF9
:1016E000BE4FBC9282E090E0D8018D939C93E75F5F
:1016F000FE4F908281E009C09394D6CFBA948ECFEA
:10170000E45DFE4F8FEF808380E0DF91CF911F91EA
:101710000F91FF90EF90DF90CF90BF90AF909F9090
:101720008F9008950F931F93CF93DF938A01E90160
:101730008AE094E00E94C717B8018AE094E00E9412
:10174000C717BE018AE094E0DF91CF911F910F91FE
:101750000C94C717EF92FF920F931F93CF93DF93D1
:10176000EC01F62EE42EB9018AE094E00E94C7173E
:10177000EF1460F0FE01EF0DF11D4AE050E06285CC
:101780008AE094E00E94E618F394F2CFB8018AE070
:1017900094E00E94C71780E0DF91CF911F910F91D5
:1017A000FF90EF90089570E0FC0126A1332727FDFC
:1017B00030956217730751F027A1332727FD309525
:1017C00081E06217730719F080E0089581E00895C1
:1017D00070E0FC0120A5332727FD309562177307C1
:1017E00051F021A5332727FD309581E0621773075B
:1017F00019F080E0089581E008959F92AF92BF9222
:10180000CF92DF92EF92FF920F931F93CF93DF93CC
:1018100000D01F92CDB7DEB78C017B0120E330E30F
:1018200040E029833A834B83FC01668DF3E06F9F90
:10183000B0011124C7010E943019E114F10449F1EB
:10184000912C87ECA82E81E0B82ECE0101966C0178
:10185000F801868D8915E8F0F80183A1981620F427
:10186000E90DF11D808101C08FEF1F928F93BF9210
:10187000AF92DF92CF920E947720B601C7010E94FB
:10188000691A93940F900F900F900F900F900F90F4
:10189000DFCF0F900F900F90DF91CF911F910F919D
:1018A000FF90EF90DF90CF90BF90AF909F90089502
:1018B0000F931F93CF93DF938C01EB0160E270E0F5
:1018C000CE010E943019209709F468C06CEC71E0D9
:1018D000CE010E94691AF80184A195A126A1220FC8
:1018E000330B820F931FFC01E15EFE4F608171811B
:1018F000CE010E94B81A6BE3CE010E94791A60ED06
:1019000071E0CE010E94691AF80184A195A127A176
:10191000220F330B820F931FFC01E15EFE4F6081AB
:101920007181CE010E94B81A6BE3CE010E94791A30
:1019300064ED71E0CE010E94691AF80184A195A1BD
:1019400020A5220F330B820F931FFC01E15EFE4F97
:1019500060817181CE010E94B81A6BE3CE010E94B2
:10196000791A68ED71E0CE010E94691AF80184A12C
:1019700095A121A5220F330B820F931FFC01E15E7D
:10198000FE4F60817181CE010E94B81A6BE3CE01D7
:10199000DF91CF911F910F910C94791ADF91CF9124
:1019A0001F910F9108950F931F93CF93DF938C0195
:1019B000EB0167E070E0CE010E943019209799F0AA
:1019C0006CED71E0CE010E94691AF80162A573A561
:1019D000CE010E94B81A6BE3CE01DF91CF911F9127
:1019E0000F910C94791ADF91CF911F910F91089567
:1019F0004F925F926F927F928F929F92AF92BF921F
:101A0000CF92DF92EF92FF920F931F93CF93DF93CA
:101A1000EC010CA11DA1580185EDA81A8EEFB80AA2
:101A2000F5018081843008F4C4C06801F8EFCF1A52
:101A3000FEEFDF0AF601608170E080E090E00E9436
:101A40002B1C2AE037ED43E25DE30E94DF1C0E947D
:101A5000FD1B40E050E0912C812CEE24EA94FE2CFA
:101A6000262F30E0F5018081481708F06BC0642F05
:101A700070E0F801E60FF71FE4818E2F992787FDAC
:101A80009095821793070CF45BC0660F771F600F69
:101A9000711FDB01A15EBE4F6D917C91161617067A
:101AA0004CF55E0F8394E60EF71EEFA1EF3F69F051
:101AB0008E2F880F990B800F911FDC01A15EBE4F06
:101AC0008D919C91861797070CF4E42FEFA3E9A55D
:101AD000EF3F69F08E2F880F990B800F911FDC016B
:101AE000A15EBE4F8D919C91681779070CF4E42F8D
:101AF000E9A726C05E1B9394EEA1EF3F69F08E2FFD
:101B0000880F990B800F911FDC01A15EBE4F8D9154
:101B10009C91681779070CF4E42FEEA3E8A5EF3F3A
:101B200069F08E2F880F990B800F911FDC01A15E49
:101B3000BE4F8D919C91861797070CF4E42FE8A770
:101B40004F5F90CF652F70E080E090E00E942B1CEB
:101B50002B013C01F601608170E080E090E00E9482
:101B60002B1C2AE037ED43EA5CE30E94DF1C9B015B
:101B7000AC01C301B2010E94DB1C1816D4F098100E
:101B800018C0C70163E070E00E94621D7BA76AA7CE
:101B90009EA19F3F71F088A58F3F59F0981749F09B
:101BA0002FA12F3F31F099A59F3F19F081E0291314
:101BB00001C080E0DF91CF911F910F91FF90EF90D6
:101BC000DF90CF90BF90AF909F908F907F906F905D
:101BD0005F904F900895FC0183A12E2FDF019A2F73
:101BE000921B981710F41D92FACF168E178E87E06D
:101BF00082A3089524E1FC0124A70C94EB0D7F92AD
:101C00008F929F92AF92BF92CF92DF92EF92FF920C
:101C10000F931F93CF93DF93EC018CA19DA1FC0147
:101C2000E45FFE4F108233971082D12CF12C812C6F
:101C300037E0B32EAA24A3940CA11DA1F801E85FFC
:101C4000FE4F8081881608F04DC0F11014C0F801D5
:101C5000E80DF11DE2846E2DCE010E94D30B81119F
:101C600006C06E2DCE010E94E80B8823C9F1F80151
:101C7000E75FFE4F80820CA11DA1D1108FC0C8016B
:101C8000885F9E4F7C01F801E80DF11DC2846C2D28
:101C9000CE010E94D30B811161C0F70180818816AB
:101CA00008F47AC05BC0672DCE010E94E80B782E45
:101CB000811184C04F8D50E02CA5332727FD30952E
:101CC000421753070CF0C8C07110B4C0CE010E9477
:101CD000EB0DF12C4E8D8BA1481708F486C0DF2C3C
:101CE0008394AACF88122DC0D801A75FBE4F4C9114
:101CF000423038F12F8D30E08CA587FD8F5F8595C0
:101D0000992787FD909582179307DCF4841A8082C7
:101D10008CA19DA1FC01E85FFE4F408150E04F5F28
:101D20005F4F3196608170E0665F7F4F680F791F6B
:101D30000A960E94DD1FECA1FDA1E45FFE4F81E049
:101D400080834F8D50E02CA5332727FD309581E00F
:101D5000421753070CF0B5C080E0B3C0282DF7013F
:101D600080818816B0F4C8018C0D911D8C0D911DD9
:101D7000FC01E15EFE4F9180991C9924991CF801A9
:101D8000E75FFE4F8080281949F020FF07C0839449
:101D900005C0FF24F394A4CF839475CFE82CF12CD5
:101DA0006801CE0CDF1CF6017284672DCE010E9403
:101DB000D30B882309F477CF9A2414C0F801E85F85
:101DC000FE4F208130E021503109E216F3060CF07D
:101DD00071CFF6016385CE010E94E80B882309F4D8
:101DE00069CF8394FF24F39475CF5AA1852F90E097
:101DF000292D332727FD3095052E01C0220F0A9487
:101E0000EAF7FE01E40FF11D3081322B30832F8D74
:101E10002F5F2F8F28A1821B910997FD03C0521BB2
:101E20005AA35DCFBAA24F5F4E8FFE01E40FF11DA2
:101E3000108255CFF801E85FFE4F808190E0019756
:101E4000E816F9060CF042CFF6016385CE010E9438
:101E5000E80B882389F13ACFF801E65FFE4F8082D4
:101E60008CA19DA1FC01E85FFE4FDC01A65FBE4F87
:101E700020818C91281B20838CA19DA1FC01E85F0F
:101E8000FE4F408150E04F5F5F4F3296608170E0BF
:101E9000665F7F4F680F791F0A960E94DD1FECA1D5
:101EA000FDA1E45FFE4F81E080834F8D50E02CA5C3
:101EB000332727FD30954CCFF801E75FFE4F808038
:101EC00005CFDF91CF911F910F91FF90EF90DF90A1
:101ED000CF90BF90AF909F908F907F9008953F924A
:101EE0004F925F926F927F928F929F92AF92BF922A
:101EF000CF92DF92EF92FF920F931F93CF93DF93D6
:101F0000CDB7DEB7E3970FB6F894DEBF0FBECDBFF7
:101F10007C013C0188EF681A8EEF780AF30180811A
:101F2000883208F474C2C7010E942D0940E060E0C5
:101F3000C7010E940D09C7010E943E0AC7010E9405
:101F4000ED0AF7018381882309F422C1EF5EFE4F79
:101F500080819181029709F01BC14701F7EF8F1A29
:101F6000FEEF9F0AF40160815701F6EFAF1AFEEF12
:101F7000BF0A82E0860FF5018083F3017081872F0D
:101F800090E00197D701A45DBE4FF5011081212F8C
:101F900030E028173907FCF4F701E20FF31F4385FF
:101FA00050E02C91332727FD30954217530779F4E1
:101FB000428550E0F7012081332727FD30954217F5
:101FC000530729F41150F501108311E005C01E5F7D
:101FD000F5011083DACF10E0F5018081781708F45D
:101FE0007083F5014081C7010E940D09112351F052
:101FF000F501808190E0F4012081821B910988978E
:1020000034F4C2C0F30140814E3F08F09EC0670126
:10201000F3EDCF1AFEEFDF0A67E072E0C6010E941F
:10202000C51987010D5C1E4F67E072E0C8010E9470
:10203000C51962E0C6010E94791A6FED71E0C60110
:102040000E94691A6BE3C6010E94791A312C37018C
:1020500085ED681A8EEF780AF3018081381640F515
:10206000432C512CF701E40DF51D84818823F1F0F8
:1020700060E5C6010E94791A632DC6010E948C1A80
:102080006DED71E0C6010E94691AC201880F991FA7
:102090008E0D9F1DFC01E15EFE4F60817181C601C6
:1020A0000E94B81A6BE3C6010E94791A3394D4CF08
:1020B00062EE71E0C6010E94691A6BE3C8010E94DA
:1020C000791A65EE71E0C8010E94691AF701608112
:1020D000772767FD7095C8010E94B81A6BE3C801A5
:1020E0000E94791A69EE71E0C8010E94691AF7012D
:1020F000E45DFE4F6081772767FD7095C8010E94FF
:10210000B81A6BE3C8010E94791AF701E35FFE4F2A
:102110008081882349F06DEE71E0C8010E94691A40
:102120006BE3C8010E94791A63E0C8010E94791A22
:102130006AE0C8010E94791A9601F5014081F40114
:102140006081C7010E94AA0BD1C0F4016081623096
:10215000D8F0F501808190E08D3F9105ACF0461BF1
:10216000F301408350E04F5F5F4F70E0665F7F4F49
:102170006E0D7F1DC7010A960E94DD1F81E0F701E9
:10218000E45FFE4F8083BBC0C7010E94A608B7C0B2
:10219000F7018181811104C08281882309F4ABC0D9
:1021A000F701EF5EFE4F80819181019709F0A3C096
:1021B000F3018081883208F49EC06701F3EDCF1AE5
:1021C000FEEFDF0A67E072E0C6010E94C5198701D1
:1021D0000D5C1E4F67E072E0C8010E94C51962E005
:1021E000C6010E94791A8EE18CA381E089A31AA20C
:1021F000CE0101960E94EB0D29A187E090E0821BA1
:1022000091097AA167E041E050E0262F30E0821783
:1022100093074CF49A01062E01C0220F0A94EAF7A4
:10222000722B6150F2CF7AA38FEF8FA388A789A773
:102230008AA7FEA2EDA2CE0101960E94FA0DCE0160
:1022400001960E94FA0D81E18DA7F7018281882312
:1022500009F45FC0CE0101960E94F80C882309F4AE
:1022600058C0CE0101960E94FF0D882309F451C089
:1022700067E072E0CE018E960E946D1962EE71E009
:10228000CE018E960E94C519BE01625D7F4FCE01C0
:1022900001960E94FD0B62EF71E0C6010E94691A6F
:1022A0006BE3C6010E94791AB601CE0101960E9425
:1022B000580C6BE3C8010E94791AB801CE0101964F
:1022C0000E94D30C63E0C8010E94791A6AE0C80139
:1022D0000E94791A9801AE01425D5F4FB601C701B5
:1022E0000E94920BCE018E960E94FF1881E0F701AA
:1022F000E55FFE4F47CFF701E55FFE4F1082F70124
:10230000E45FFE4F8081811182C0C7010E94A60850
:102310007EC0F7018181882349F36FEE71E0C60129
:102320000E94691A6BE3C6010E94791A512C570169
:10233000F5EDAF1AFEEFBF0AF5018081581648F59A
:10234000852C912CF701E80DF91D84818823F9F083
:1023500060EC71E0C6010E94691A652DC6010E94F9
:102360008C1A6DED71E0C6010E94691AC401880FD4
:10237000991F8E0D9F1DFC01E15EFE4F60817181F2
:10238000C6010E94B81A6BE3C6010E94791A5394E1
:10239000D3CF62EE71E0C6010E94691A6BE3C801F7
:1023A0000E94791A65EE71E0C8010E94691AF7016E
:1023B0006081772767FD7095C8010E94B81A6BE3AA
:1023C000C8010E94791AF701E35FFE4F80818823DC
:1023D00049F06DEE71E0C8010E94691A6BE3C80113
:1023E0000E94791A63E0C8010E94791A6AE0C80164
:1023F0000E94791AF30140814150960160E0C701C3
:102400000E94AA0BF701E45FFE4F10826FCFE396A4
:102410000FB6F894DEBF0FBECDBFDF91CF911F91F5
:102420000F91FF90EF90DF90CF90BF90AF909F9073
:102430008F907F906F905F904F903F9008958F9214
:102440009F92AF92BF92CF92DF92EF92FF920F9343
:102450001F93CF93DF931F92CDB7DEB74C018C0152
:10246000085F1E4FD8018C9190E08D3F910544F09C
:1024700081E0F401E35FFE4F8083C4010E946F0F8F
:10248000F401E05FFE4F10826401B9EECB1ABEEF9B
:10249000DB0AD601ED91FC91119780819181129612
:1024A0000D90BC91A02D2D913C91D8014C91509153
:1024B00000047401B5EDEB1ABEEFFB0AD7016C9175
:1024C000651708F45C93442361F082279327B92EA3
:1024D000BB1CBB24BB1C81E04D3F09F480E0B8224B
:1024E00005C0D7011C9210920004B12C608171814B
:1024F000C40149830E94E708A82E498187FD2CC0AA
:10250000F401E40FF11D8287423030F081858A1199
:1025100003C0C4010E94A6088A2D880F990B880D5C
:10252000991DFC01E15EFE4FD6018D919C912081A9
:102530003181DC018D919C91280F391F37FF02C03A
:102540002F5F3F4F3595279531832083F801808198
:102550008F5F808320E012C040E060E0C4010E94F1
:102560000D09D7018C91863041F480910004F4016B
:10257000E80FF11D8481823024F421E0B1101DC0E8
:1025800001C020E0F8018081A401455F5E4F5A013F
:10259000883248F081E0DA018C93C4010E946F0F09
:1025A000109200046AC0C40129830E94A608F501A4
:1025B00010821092000429810BC0D8018C918832BE
:1025C00038F083E090E0F401EF5EFE4F918380836A
:1025D000222309F452C0F80140815091000480E0A8
:1025E00090E0242F30E0F9013197280D391DBF010B
:1025F000680F791F6F3FAFEF7A07E1F00197D901BC
:10260000A80FB91F1A96AC91A513F1CFCB01019673
:10261000481BD8014C9350E04F5F5F4F655F7F4F81
:10262000680D791DC4010A960E94DD1FF8018081A2
:102630008F5F808340910004D601ED91FC91208151
:102640003181C401840F911D840F911DFC01E15E55
:10265000FE4F31832083F8018081F401E80FF11DE2
:1026600042878F5FD8018C934F5F409300044630C0
:1026700021F410920004F70140830F90DF91CF9175
:102680001F910F91FF90EF90DF90CF90BF90AF9090
:102690009F908F900895CF93DF93EC01C55FDE4F3D
:1026A0001882FC01E75EFE4F0190F081E02D208151
:1026B0003181DC01A95EBE4F0D90BC91A02D2D9300
:1026C0003C93DB012D913C91318320830E941F12AA
:1026D0008881DF91CF91089508958230E8F4E82F42
:1026E000F0E0EE0FFF1FE75FFE4F718360838130E4
:1026F00041F0809169008C7F842B80936900E89A77
:10270000089580916900440F551F440F551F837F22
:10271000842B80936900E99A0895823078F481309F
:1027200011F0E89801C0E998E82FF0E0EE0FFF1FE4
:10273000E75FFE4F8CE693E19183808308951F92BB
:102740000F920FB60F9211242F933F934F935F93E5
:102750006F937F938F939F93AF93BF93EF93FF9369
:10276000E0910901F0910A010995FF91EF91BF9164
:10277000AF919F918F917F916F915F914F913F9119
:102780002F910F900FBE0F901F9018951F920F92D0
:102790000FB60F9211242F933F934F935F936F9334
:1027A0007F938F939F93AF93BF93EF93FF93E091AA
:1027B0000B01F0910C010995FF91EF91BF91AF9141
:1027C0009F918F917F916F915F914F913F912F9149
:1027D0000F900FBE0F901F9018951F920F920FB67B
:1027E0000F9211242F933F938F939F93AF93BF9397
:1027F0008091020490910304A0910404B091050417
:102800003091010423E0230F2D3720F40196A11D00
:10281000B11D05C026E8230F0296A11DB11D20930E
:1028200001048093020490930304A0930404B093E2
:1028300005048091060490910704A0910804B091CA
:1028400009040196A11DB11D80930604909307040D
:10285000A0930804B0930904BF91AF919F918F9109
:102860003F912F910F900FBE0F901F9018952FB78B
:10287000F894609102047091030480910404909193
:1028800005042FBF08953FB7F894809106049091F6
:102890000704A0910804B091090426B5A89B05C0BF
:1028A0002F3F19F00196A11DB11D3FBF6627782F5C
:1028B000892F9A2F620F711D811D911D42E0660FB5
:1028C000771F881F991F4A95D1F70895CF92DF92FD
:1028D000EF92FF92CF93DF936B017C010E94431430
:1028E000EB01C114D104E104F10489F00E94921BB0
:1028F0000E9443146C1B7D0B683E734090F381E093
:10290000C81AD108E108F108C851DC4FEACFDF91BD
:10291000CF91FF90EF90DF90CF9008958230910596
:1029200038F0880F991F880F991F05970197F1F7C5
:102930000895789484B5826084BD84B5816084BD37
:1029400085B5826085BD85B5816085BDEEE6F0E028
:10295000808181608083E1E8F0E010828081826084
:102960008083808181608083E0E8F0E08081816005
:102970008083E1EBF0E0808184608083E0EBF0E035
:10298000808181608083EAE7F0E0808184608083D9
:102990008081826080838081816080838081806883
:1029A00080831092C1000895833081F028F4813033
:1029B00099F08230A1F008958730A9F08830B9F0FD
:1029C0008430D1F4809180008F7D03C0809180009D
:1029D0008F7780938000089584B58F7702C084B587
:1029E0008F7D84BD08958091B0008F7703C0809162
:1029F000B0008F7D8093B0000895CF93DF9390E077
:102A0000FC01E555FF4F2491FC01E154FF4F8491F7
:102A1000882349F190E0880F991FFC01E352FF4F92
:102A2000A591B4918D529F4FFC01C591D4919FB750
:102A3000611108C0F8948C91209582238C93888131
:102A400082230AC0623051F4F8948C91322F309571
:102A500083238C938881822B888304C0F8948C9183
:102A6000822B8C939FBFDF91CF9108950F931F937B
:102A7000CF93DF931F92CDB7DEB7282F30E0F90157
:102A8000E956FF4F8491F901E555FF4F1491F90183
:102A9000E154FF4F04910023C9F0882321F069839A
:102AA0000E94D4146981E02FF0E0EE0FFF1FED5279
:102AB000FF4FA591B4919FB7F8948C91611103C019
:102AC0001095812301C0812B8C939FBF0F90DF91C4
:102AD000CF911F910F910895FC01818D228D90E07F
:102AE000805C9F4F821B91098F7399270895FC0189
:102AF000918D828D981731F0828DE80FF11D858DB3
:102B000090E008958FEF9FEF0895FC01918D828DE5
:102B1000981761F0828DDF01A80FB11D5D968C9131
:102B2000928D9F5F9F73928F90E008958FEF9FEF3C
:102B3000089589E097E1892B49F08EE598E0892B8B
:102B400029F00E94091781110C945E080895FC0178
:102B5000848DDF01A80FB11DA35ABF4F2C91848D26
:102B600090E001968F739927848FA689B7892C935B
:102B7000A089B1898C9180648C93938D848D9813F6
:102B800006C00288F389E02D80818F7D80830895BF
:102B9000CF93DF93EC01888D8823C9F0EA89FB8904
:102BA000808185FD05C0A889B9898C9186FD0FC0FB
:102BB0000FB607FCF5CF808185FFF2CFA889B989D0
:102BC0008C9185FFEDCFCE010E94A715E7CFDF9155
:102BD000CF910895CF92DF92FF920F931F93CF93DF
:102BE000DF931F92CDB7DEB76C0181E0D601589616
:102BF0008C9358975B969C915B975C968C915C97B5
:102C0000981307C05096ED91FC915197808185FDF6
:102C10002EC0F601038D10E00F5F1F4F0F731127B9
:102C2000F02EF601848DF81211C00FB607FCF9CF13
:102C3000D6015096ED91FC915197808185FFF1CF9F
:102C4000C60169830E94A7156981EBCF838DE80FC8
:102C5000F11DE35AFF4F6083D6015B960C935B979F
:102C60005296ED91FC915397808180620CC0D60101
:102C70005696ED91FC91579760835096ED91FC919B
:102C8000519780818064808381E090E00F90DF9194
:102C9000CF911F910F91FF90DF90CF900895BF9239
:102CA000CF92DF92EF92FF92CF93DF93EC016A0114
:102CB0007B01B22EE889F98982E08083411581EE9B
:102CC000580761057105A1F060E079E08DE390E0BF
:102CD000A70196010E94761D215031094109510931
:102CE0005695479537952795211580E1380798F037
:102CF000E889F989108260E874E88EE190E0A70124
:102D000096010E94761D21503109410951095695BD
:102D1000479537952795EC85FD853083EE85FF85B2
:102D20002083188EEC89FD89B082EA89FB89808135
:102D300080618083EA89FB89808188608083EA8959
:102D4000FB89808180688083EA89FB8980818F7D0F
:102D50008083DF91CF91FF90EF90DF90CF90BF9075
:102D600008951F920F920FB60F9211242F938F93F5
:102D70009F93EF93FF93E0911A04F0911B048081DD
:102D8000E0912004F091210482FD12C09081809195
:102D900023048F5F8F7320912404821751F0E091F8
:102DA0002304F0E0E65FFB4F958F8093230401C07E
:102DB0008081FF91EF919F918F912F910F900FBE86
:102DC0000F901F9018951F920F920FB60F9211241B
:102DD0002F933F934F935F936F937F938F939F9323
:102DE000AF93BF93EF93FF938AE094E00E94A715FF
:102DF000FF91EF91BF91AF919F918F917F916F91D3
:102E00005F914F913F912F910F900FBE0F901F90A8
:102E100018958AE094E00E946C1521E0892B09F452
:102E200020E0822F089510920D0410920C0488EE79
:102E300093E0A0E0B0E080930E0490930F04A09381
:102E40001004B093110489EF91E090930B048093E8
:102E50000A0485EC90E0909317048093160484ECA8
:102E600090E0909319048093180480EC90E0909384
:102E70001B0480931A0481EC90E090931D048093CE
:102E80001C0482EC90E090931F0480931E0486EC57
:102E900090E09093210480932004109223041092D8
:102EA00024041092250410922604089508950E9487
:102EB00099140E9456170E94C507C9E9D5E10E94DE
:102EC00056072097E1F30E949915F9CFCF92DF9230
:102ED000EF92FF920F931F93CF93DF937C016A01D0
:102EE000EB0100E010E00C151D0571F06991D701B0
:102EF000ED91FC910190F081E02DC7010995892B9E
:102F000019F00F5F1F4FEFCFC801DF91CF911F91D5
:102F10000F91FF90EF90DF90CF90089561157105AC
:102F200081F0DB010D900020E9F7AD01415051091E
:102F3000461B570BDC01ED91FC910280F381E02DE3
:102F4000099480E090E00895EF92FF920F931F9311
:102F5000CF93DF938C017B01C0E0D0E0F701EC0F51
:102F6000FD1F6491662359F0F801A081B181ED91B4
:102F7000FC91C8010995892B11F02196EFCFCE0164
:102F8000DF91CF911F910F91FF90EF900895DC0199
:102F9000ED91FC91DB0114964D915C9115976D912B
:102FA0007C910280F381E02D0994DC01ED91FC918C
:102FB0000190F081E02D099465E072E00C948E1789
:102FC0000F931F93CF93DF93EC010E94A4178C0102
:102FD000CE010E94DC17800F911FDF91CF911F91CE
:102FE0000F9108950F931F93CF93DF93EC010E94ED
:102FF000C7178C01CE010E94DC17800F911FDF9153
:10300000CF911F910F9108950F931F93CF93DF934B
:10301000EC010E948E178C01CE010E94DC17800FFC
:10302000911FDF91CF911F910F9108958F929F92E1
:10303000AF92BF92CF92DF92EF92FF920F931F93C6
:10304000CF93DF93CDB7DEB7A1970FB6F894DEBF6D
:103050000FBECDBF7C01C42EE52FCB01D22E19A20D
:1030600021E02D1510F02AE0D22E8E010F5D1F4FAA
:103070008D2C912CA12CB12C6C2D7E2FA5019401AF
:103080000E94761D8C2DD29E8019112401501109A9
:103090008A3014F4805D01C0895CF80180832115B9
:1030A00031054105510521F0C22EE32FCA01E4CFBD
:1030B000B801C7010E948E17A1960FB6F894DEBF23
:1030C0000FBECDBFDF91CF911F910F91FF90EF9079
:1030D000DF90CF90BF90AF909F908F900895CF9248
:1030E000DF92EF92FF920F931F93CF93DF93EC0148
:1030F0006A017B012115310579F4E881F98101909C
:10310000F081E02D642FDF91CF911F910F91FF90FF
:10311000EF90DF90CF9009942A303105E9F477FFE2
:103120001AC06DE20E94D5178C0144275527BA01B9
:103130004C195D096E097F092AE0CE010E9416181C
:10314000800F911FDF91CF911F910F91FF90EF9012
:10315000DF90CF9008952AE0B701A601CE01DF915C
:10316000CF911F910F91FF90EF90DF90CF900C9433
:1031700016189A01AB01662757FD6095762F0C94BF
:103180006F180F931F93CF93DF93EC019A01AB015C
:10319000662757FD6095762F0E946F188C01CE012F
:1031A0000E94DC17800F911FDF91CF911F910F912B
:1031B00008952115310541F4DC01ED91FC91019058
:1031C000F081E02D642F09940C9416189A01462F73
:1031D00050E060E070E00C94D9180F931F93CF93E8
:1031E000DF93EC010E94D9188C01CE010E94DC17FC
:1031F000800F911FDF91CF911F910F910895FC01D6
:10320000808191810C94361ECF93DF93EC018881ED
:103210009981009711F00E94361E198218821D8232
:103220001C821B821A82DF91CF9108950F931F9306
:10323000CF93DF93EC018B016F5F7F4F8881998182
:103240000E94C51E009731F0998388831B830A83EF
:1032500081E001C080E0DF91CF911F910F9108952F
:10326000CF93DF93EC0188819981892B29F08A81A2
:103270009B818617970760F4CE010E941619882358
:1032800041F08C819D81892B19F4E881F9811082AC
:1032900081E0DF91CF910895EF92FF920F931F93FA
:1032A000CF93DF93EC017B018A01BA010E943019B0
:1032B000811104C0CE010E94041907C01D830C8334
:1032C000B701888199810E94EF1FCE01DF91CF91D4
:1032D0001F910F91FF90EF900895FC0111821082D1
:1032E00013821282158214826115710559F0FB0157
:1032F00001900020E9F7AF0141505109461B570BDF
:103300000C944C1908950F931F93CF93DF938C0166
:10331000EB01FC0180819181009799F042815381FA
:103320002C813D814217530750F0688179810E94BA
:10333000EF1F8C819D81F8019583848313C00E94C7
:10334000361E88819981F801918380838A819B81CF
:10335000938382838C819D819583848319821882D3
:103360001B821A821D821C82DF91CF911F910F91C7
:103370000895CF93DF93EC018617970711F00E9411
:103380008319CE01DF91CF910895CF93DF93EC01A4
:103390006115710561F0FB0101900020E9F7AF01B3
:1033A00041505109461B570B0E944C1902C00E9404
:1033B0000419CE01DF91CF9108950F931F93CF93FE
:1033C000DF93CDB7DEB729970FB6F894DEBF0FBEF7
:1033D000CDBF8C01862FF8011182108213821282D8
:1033E0001582148250E0BE016F5F7F4F90E00E9413
:1033F0005220BE016F5F7F4FC8010E94C5192996F8
:103400000FB6F894DEBF0FBECDBFDF91CF911F91F5
:103410000F9108950F931F93CF93DF93CDB7DEB72E
:1034200062970FB6F894DEBF0FBECDBF8C01CB0103
:10343000F80111821082138212821582148250E0E8
:10344000BE016F5F7F4F0E941F20BE016F5F7F4FE5
:10345000C8010E94C51962960FB6F894DEBF0FBE70
:10346000CDBFDF91CF911F910F910895EF92FF9201
:103470000F931F93CF93DF93EC017B010C811D8190
:103480006115710511F480E016C04115510591F0E8
:10349000040F151FB8010E9430198823A1F3288159
:1034A00039818C819D81B701820F931F0E94EF1F8C
:1034B0001D830C8381E0DF91CF911F910F91FF90CD
:1034C000EF900895FB0144815581608171810C94D6
:1034D000361A6115710559F0FB0101900020E9F7DA
:1034E000AF0141505109461B570B0C94361A80E02E
:1034F0000895CF93DF9300D0CDB7DEB769831A82EA
:1035000041E050E0BE016F5F7F4F0E94361A0F907E
:103510000F90DF91CF910895EF92FF920F931F9339
:10352000CF93DF9300D000D0CDB7DEB77C01862FDC
:103530004AE08E010F5F1F4FB80190E00E942A20E1
:10354000F80101900020E9F7AF0141505109401BFB
:10355000510BB801C7010E94361A0F900F900F90BF
:103560000F90DF91CF911F910F91FF90EF900895F1
:10357000EF92FF920F931F93CF93DF93CDB7DEB7F8
:1035800028970FB6F894DEBF0FBECDBF7C01CB01EC
:103590004AE08E010F5F1F4FB8010E942A20F801F8
:1035A00001900020E9F7AF0141505109401B510B38
:1035B000B801C7010E94361A28960FB6F894DEBFEC
:1035C0000FBECDBFDF91CF911F910F91FF90EF9074
:1035D0000895FC01248135816217730748F48081C6
:1035E0009181009729F0FC01E60FF71F8081089573
:1035F00080E008950C94E91A0F931F93CF93DF9303
:10360000EB0141155105E9F02097D9F0FC016481E7
:10361000758126173707A0F4621B730B8A010150CE
:1036200011096017710708F48B01FC016081718139
:10363000620F731FA801CE010E94F61FC00FD11F99
:103640001882DF91CF911F910F910895CF93DF934F
:10365000FC01848195814817590778F4C081D18194
:10366000FB0160817181CE01840F951F0E940520AE
:10367000009719F08C1B9D0B02C08FEF9FEFDF911D
:10368000CF910895BF92CF92DF92EF92FF920F9366
:103690001F93CF93DF936C017B01EA01890124170B
:1036A000350720F48D2FE901042F182F67E072E011
:1036B000C6010E946D19D70114968D919C911597A2
:1036C000C817D907C8F48017910708F48C01D701EF
:1036D000ED91FC911197E00FF11FB08010826D9178
:1036E0007C916C0F7D1FC6010E94C519D701ED9119
:1036F000FC91E00FF11FB082C601DF91CF911F91C5
:103700000F91FF90EF90DF90CF90BF900895FC0154
:1037100080819181009711F00C94AD1F60E070E002
:10372000CB01089508955058BB27AA270ED009C190
:10373000FAD030F0FFD020F031F49F3F11F41EF4A6
:10374000EFC00EF4E095E7FBE5C0E92F0BD180F365
:10375000BA17620773078407950718F071F49EF58E
:1037600023C10EF4E0950B2EBA2FA02D0B01B90149
:1037700090010C01CA01A0011124FF27591B99F0E7
:10378000593F50F4503E68F11A16F040A22F232FF3
:10379000342F4427585FF3CF469537952795A79543
:1037A000F0405395C9F77EF41F16BA0B620B730BEA
:1037B000840BBAF09150A1F0FF0FBB1F661F771F5B
:1037C000881FC2F70EC0BA0F621F731F841F48F410
:1037D000879577956795B795F7959E3F08F0B3CF96
:1037E0009395880F08F09927EE0F97958795089580
:1037F00004D06894B111D9C00895BCD088F09F5707
:1038000090F0B92F9927B751A0F0D1F0660F771F2C
:10381000881F991F1AF0BA95C9F712C0B13081F00C
:10382000C3D0B1E00895C0C0672F782F8827B85F54
:1038300039F0B93FCCF3869577956795B395D9F76D
:103840003EF490958095709561957F4F8F4F9F4F77
:103850000895E89409C097FB3EF490958095709583
:1038600061957F4F8F4F9F4F9923A9F0F92F96E9CC
:10387000BB279395F695879577956795B795F11141
:10388000F8CFFAF4BB0F11F460FF1BC06F5F7F4FDE
:103890008F4F9F4F16C0882311F096E911C07723F0
:1038A00021F09EE8872F762F05C0662371F096E8F9
:1038B000862F70E060E02AF09A95660F771F881FC8
:1038C000DAF7880F9695879597F90895990F00086C
:1038D000550FAA0BE0E8FEEF16161706E807F907E2
:1038E000C0F012161306E407F50798F0621B730B7D
:1038F000840B950B39F40A2661F0232B242B252BFE
:1039000021F408950A2609F4A140A6958FEF811DA0
:10391000811D089597F99F6780E870E060E0089541
:103920009FEF80EC089500240A94161617061806D7
:103930000906089500240A941216130614060506B3
:103940000895092E0394000C11F4882352F0BB0F44
:1039500040F4BF2B11F460FF04C06F5F7F4F8F4FA7
:103960009F4F089557FD9058440F551F59F05F3FE2
:1039700071F04795880F97FB991F61F09F3F79F091
:1039800087950895121613061406551FF2CF469513
:10399000F1DF08C0161617061806991FF1CF869595
:1039A0007105610508940895E894BB276627772779
:1039B000CB0197F908958ADF08F48FEF08950BD0B3
:1039C000C0CFB1DF28F0B6DF18F0952309F0A2CF01
:1039D000A7CF1124EACFC6DFA0F3959FD1F3950FAF
:1039E00050E0551F629FF001729FBB27F00DB11D83
:1039F000639FAA27F00DB11DAA1F649F6627B00D13
:103A0000A11D661F829F2227B00DA11D621F739FFB
:103A1000B00DA11D621F839FA00D611D221F749F09
:103A20003327A00D611D231F849F600D211D822F50
:103A3000762F6A2F11249F5750408AF0E1F0882397
:103A40004AF0EE0FFF1FBB1F661F771F881F9150A4
:103A50005040A9F79E3F510570F05CCFA6CF5F3F65
:103A6000ECF3983EDCF3869577956795B795F795D7
:103A7000E7959F5FC1F7FE2B880F911D969587955F
:103A800097F90895991B79E004C0991F961708F0DB
:103A9000961B881F7A95C9F780950895AA1BBB1BB2
:103AA00051E107C0AA1FBB1FA617B70710F0A61B3E
:103AB000B70B881F991F5A95A9F780959095BC015F
:103AC000CD01089597FB072E16F4009407D077FDDB
:103AD00009D00E944E1D07FC05D03EF490958195BB
:103AE0009F4F0895709561957F4F0895A1E21A2E1A
:103AF000AA1BBB1BFD010DC0AA1FBB1FEE1FFF1F92
:103B0000A217B307E407F50720F0A21BB30BE40BE1
:103B1000F50B661F771F881F991F1A9469F7609528
:103B20007095809590959B01AC01BD01CF010895E2
:103B3000EE0FFF1F0590F491E02D0994CF93DF93D2
:103B40008230910510F482E090E0E091A904F091B8
:103B5000AA0420E030E0A0E0B0E0309739F14081E5
:103B6000518148175907B8F04817590771F48281F5
:103B70009381109729F013969C938E9312972CC0E3
:103B80009093AA048093A90427C02115310531F030
:103B90004217530718F0A901DB0101C0EF019A0198
:103BA000BD01DF010280F381E02DD7CF2115310562
:103BB000F9F0281B390B2430310580F48A819B8170
:103BC0006115710521F0FB019383828304C09093FA
:103BD000AA048093A904FE01329644C0FE01E20FBC
:103BE000F31F8193919322503109398328833AC07E
:103BF0002091A7043091A804232B41F420910201C5
:103C0000309103013093A8042093A7042091000170
:103C1000309101012115310541F42DB73EB7409196
:103C2000040150910501241B350BE091A704F0918C
:103C3000A804E217F307A0F42E1B3F0B281739073F
:103C400078F0AC014E5F5F4F2417350748F04E0FF8
:103C50005F1F5093A8044093A7048193919302C0DF
:103C6000E0E0F0E0CF01DF91CF910895CF93DF93B3
:103C7000009709F487C0FC01329713821282C09129
:103C8000A904D091AA04209781F420813181280FC2
:103C9000391F8091A7049091A8048217930779F5A2
:103CA000F093A804E093A7046DC0DE0120E030E0AB
:103CB000AE17BF0750F412964D915C9113979D017A
:103CC0004115510509F1DA01F3CFB383A283408195
:103CD0005181840F951F8A179B0771F48D919C91D8
:103CE0001197840F951F02969183808312968D9170
:103CF0009C911397938382832115310529F4F093C6
:103D0000AA04E093A9043EC0D9011396FC93EE9354
:103D100012974D915D91A40FB51FEA17FB0779F437
:103D200080819181840F951F0296D90111969C93F1
:103D30008E938281938113969C938E931297E0E0E9
:103D4000F0E08A819B81009719F0FE01EC01F9CF28
:103D5000CE01029628813981820F931F2091A704FA
:103D60003091A8042817390769F4309729F4109284
:103D7000AA041092A90402C013821282D093A8044C
:103D8000C093A704DF91CF910895A0E0B0E0EBECE1
:103D9000FEE10C943B23EC01CB01209719F40E9427
:103DA0009E1DB8C0FE01E60FF71F9E01225031098B
:103DB000E217F30708F4ACC0D9010D911C911197DB
:103DC00006171707B8F00530110508F49FC0A801C1
:103DD000445051094617570708F498C0025011097A
:103DE000061B170B019311936D937C93CF010E94D7
:103DF000361E8CC05B01A01AB10A4E01800E911EC6
:103E0000A091A904B091AA04612C712C60E070E02B
:103E1000109709F449C0A815B905C9F5ED90FC90B3
:103E20001197670142E0C40ED11CCA14DB0478F17B
:103E300047018A189B08640142E0C40ED11C129607
:103E4000BC9012971396AC91B5E0CB16D10440F01C
:103E5000B282A38391828082D9018D939C9309C001
:103E60000E5F1F4F0E0D1F1DF90111830083EB2DF7
:103E7000FA2F6115710531F0DB011396FC93EE9377
:103E8000129744C0F093AA04E093A9043FC06D9137
:103E90007C9111976616770608F43B01BD011296D6
:103EA0000D90BC91A02DB4CF6091A7047091A8048F
:103EB00068157905E9F468167906D0F44091000197
:103EC000509101014115510541F44DB75EB7609124
:103ED000040170910501461B570BE417F507C0F468
:103EE000F093A804E093A704F901918380830EC0A6
:103EF0000E949E1D7C01009759F0A801BE010E94FE
:103F0000D41FCE010E94361EC70104C0CE0102C0DC
:103F100080E090E0CDB7DEB7EEE00C945723FC01D3
:103F200088279927E89421912032E9F3293010F06D
:103F30002E30C8F32B3241F02D3239F4689404C08E
:103F40000E944A20820F911D219120532A30C0F3F4
:103F50001EF4909581959F4F08951F93FC0199271A
:103F60008827BC01E89411911032E9F3193010F060
:103F70001E30C8F31B3251F01D3249F4689406C05C
:103F80000E943520610F711D811D911D11911053EB
:103F90001A30B0F33EF490958095709561957F4FFF
:103FA0008F4F9F4F1F910895FB01DC0102C00190CC
:103FB0000D9241505040D8F708956817790768F47A
:103FC000FB01DC01E40FF51FA40FB51F02C0029036
:103FD0000E9241505040D8F708950C94D41FFB0125
:103FE000DC0101900D920020E1F70895FB01DC0156
:103FF0004150504048F001900D920020C9F701C097
:104000001D9241505040E0F70895FB015191552316
:10401000A9F0BF01DC014D9145174111E1F759F4B9
:10402000CD010190002049F04D9140154111C9F397
:10403000FB014111EFCF81E090E0019708954532F7
:10404000510520F4423010F00C942A20FB0110821C
:10405000CB010895BB274A3031F4992322F4BDE205
:10406000909581959F4F0C945E20592F482F372FA4
:10407000262F660F771F881F991F660F771F881FCF
:10408000991F620F731F841F951F660F771F881F6C
:10409000991F08957AE0979F902D879F802D910D0D
:1040A000112408954532510520F4423010F00C944B
:1040B0005D20FB011082CB010895BB27FB01552732
:1040C000AA27880F991FAA1FA41710F0A41B839575
:1040D0005051B9F7A05DAA3308F0A95DA1930097EC
:1040E00079F7B111B1931192CB010C949722AEE004
:1040F000B0E0EDE7F0E20C9445230D891E8986E0DF
:104100008C831A8309838FEF9FE79E838D83AE0193
:10411000475E5F4F6F89788DCE0101960E9499208E
:10412000EF81F885E00FF11F10822E96E4E00C94E9
:104130006123ACE0B0E0EFE9F0E20C9437237C01BE
:104140006B018A01FC0117821682838181FFBDC148
:10415000CE0101964C01F7019381F60193FD859103
:1041600093FF81916F01882309F4ABC1853239F443
:1041700093FD859193FF81916F01853229F4B701F9
:1041800090E00E94A722E7CF512C312C20E0203272
:10419000A0F48B3269F030F4803259F0833269F444
:1041A00020612CC08D3239F0803339F4216026C073
:1041B0002260246023C0286021C027FD27C030ED85
:1041C000380F3A3078F426FF06C0FAE05F9E300DD3
:1041D0001124532E13C08AE0389E300D1124332E43
:1041E00020620CC08E3221F426FD6BC1206406C013
:1041F0008C3611F4206802C0883641F4F60193FD34
:10420000859193FF81916F018111C1CF982F9F7D7F
:104210009554933028F40C5F1F4FFFE3F9830DC0D2
:10422000833631F0833771F0833509F05BC022C0EB
:10423000F801808189830E5F1F4F44244394512CE1
:10424000540115C03801F2E06F0E711CF801A08016
:10425000B18026FF03C0652D70E002C06FEF7FEFD5
:10426000C5012C870E948C222C0183012C852F777D
:10427000222E17C03801F2E06F0E711CF801A080E9
:10428000B18026FF03C0652D70E002C06FEF7FEFA5
:10429000C5012C870E9481222C012C852068222EAA
:1042A000830123FC1BC0832D90E048165906B0F40F
:1042B000B70180E290E00E94A7223A94F4CFF50182
:1042C00027FC859127FE81915F01B70190E00E9454
:1042D000A72231103A94F1E04F1A510841145104C9
:1042E00071F7E5C0843611F0893639F5F80127FFFA
:1042F00007C060817181828193810C5F1F4F08C06C
:1043000060817181882777FD8095982F0E5F1F4F00
:104310002F76B22E97FF09C0909580957095619584
:104320007F4F8F4F9F4F2068B22E2AE030E0A401CC
:104330000E94D922A82EA81844C0853729F42F7EC0
:10434000B22E2AE030E025C0F22FF97FBF2E8F3643
:10435000C1F018F4883579F0B4C0803719F0883787
:1043600021F0AFC02F2F2061B22EB4FE0DC08B2DD7
:104370008460B82E09C024FF0AC09F2F9660B92E12
:1043800006C028E030E005C020E130E002C020E1B6
:1043900032E0F801B7FE07C06081718182819381AC
:1043A0000C5F1F4F06C06081718180E090E00E5F5E
:1043B0001F4FA4010E94D922A82EA818FB2DFF7719
:1043C000BF2EB6FE0BC02B2D2E7FA51450F4B4FECD
:1043D0000AC0B2FC08C02B2D2E7E05C07A2C2B2DD6
:1043E00003C07A2C01C0752C24FF0DC0FE01EA0D1C
:1043F000F11D8081803311F4297E09C022FF06C09F
:104400007394739404C0822F867809F0739423FD0B
:1044100013C020FF06C05A2C731418F4530C5718FD
:10442000732C731468F4B70180E290E02C870E942B
:10443000A72273942C85F5CF731410F4371801C09C
:10444000312C24FF12C0B70180E390E02C870E943A
:10445000A7222C8522FF17C021FF03C088E590E02A
:1044600002C088E790E0B7010CC0822F867859F02F
:1044700021FD02C080E201C08BE227FD8DE2B70181
:1044800090E00E94A722A51438F4B70180E390E0E1
:104490000E94A7225A94F7CFAA94F401EA0DF11DC5
:1044A0008081B70190E00E94A722A110F5CF3320B0
:1044B00009F451CEB70180E290E00E94A7223A941D
:1044C000F6CFF7018681978102C08FEF9FEF2C9680
:1044D000E2E10C945323F999FECF92BD81BDF89A85
:1044E000992780B50895262FF999FECF1FBA92BD5E
:1044F00081BD20BD0FB6F894FA9AF99A0FBE0196C5
:104500000895FC010590615070400110D8F7809526
:1045100090958E0F9F1F0895FC016150704001908F
:104520000110D8F7809590958E0F9F1F0895DC019C
:10453000FC01672F71917723E1F7329704C07C91DA
:104540006D9370836291AE17BF07C8F308950F9300
:104550001F93CF93DF93182F092FEB018B8181FDE0
:1045600003C08FEF9FEF20C082FF10C04E815F819C
:104570002C813D81421753077CF4E881F9819F012A
:104580002F5F3F4F39832883108306C0E885F98564
:10459000812F0995892B29F72E813F812F5F3F4F6E
:1045A0003F832E83812F902FDF91CF911F910F9109
:1045B0000895FA01AA27283051F1203181F1E894B9
:1045C0006F936E7F6E5F7F4F8F4F9F4FAF4FB1E006
:1045D0003ED0B4E03CD0670F781F891F9A1FA11D01
:1045E000680F791F8A1F911DA11D6A0F711D811D02
:1045F000911DA11D20D009F468943F912AE0269FC7
:1046000011243019305D3193DEF6CF010895462F25
:104610004770405D4193B3E00FD0C9F7F6CF462F06
:104620004F70405D4A3318F0495D31FD405241936F
:1046300002D0A9F7EACFB4E0A6959795879577952C
:104640006795BA95C9F700976105710508959B01B3
:10465000AC010A2E06945795479537952795BA953C
:10466000C9F7620F731F841F951FA01D08952F9215
:104670003F924F925F926F927F928F929F92AF92F2
:10468000BF92CF92DF92EF92FF920F931F93CF933F
:10469000DF93CDB7DEB7CA1BDB0B0FB6F894DEBFD6
:1046A0000FBECDBF09942A88398848885F846E84FC
:1046B0007D848C849B84AA84B984C884DF80EE8046
:1046C000FD800C811B81AA81B981CE0FD11D0FB64F
:1046D000F894DEBF0FBECDBFED01089510E0CCEE23
:1046E000D0E004C0FE010E949A1D2296CE3ED10762
:0646F000C9F7F894FFCFAA
:1046F6000000AB0480002C01066C136C133B0049D0
:1047060054506172616D733A20004F4B005620334E
:104716002E322E302D623132205349474E414C64A1
:1047260075696E6F202D20636F6D70696C656420EE
:1047360061742046656220313320323031362032B2
:10474600313A33343A30390053796E633A200020D7
:104756002D3E2053796E63466163743A20002C2007
:10476600436C6F636B3A20002C20546F6C3A200028
:104776002C20506174744C656E3A20002C205075C4
:104786006C73653A20002C20002C206D53746172E6
:10479600743A20005369676E616C3A20002E20003F
:1047A600205B005D005061747465726E3A200020D3
:1047B60050002A5B002C0025303258004C4C3D003E
:1047C6004C483D00534C3D0053483D00433D004D91
:1047D6005300443D0043503D0053503D004F004DB3
:1047E60055004D430000000000EA1566176C15855C
:1047F600157715C8150D0A006E616E00696E6600A4
:064806006F7666002E0033
:00000001FF
